:02000000800B73
:20000B002106758127758902758C2275A882752500752600752240E590F454E0F521D2B589
:20002B00C2B1D2B211ABC2B4D28CE525B40CFB752500E590F4541FB524F0E523A200B002CE
:20004B004050A202B000404AB4100DE521B4FF02803A052111AB8034B4110AE521602D15D4
:20006B002111AB8027B41A028003B4200DE522B480028018052211AB8012B41B028003B46B
:20008B00210AE5226006152211AB8000A20092028098B40C04B2B480F3B40DACB2B580EC1F
:2000AB00C2B2E5211200EAE522B44004D2B38002C2B3C39440500EAB21E5228521F01200D4
:2000CB00F8ACF0800FAC217480C395228521F01200F8ABF0EC1200EAEB1200EAD2B2227A8D
:2000EB00083392B000D2B100C2B1DAF522A433C5F033C5F033C5F033C5F022C0E0C0D0C03B
:20010B0082C08390015FA2B7B3E5263393F526B4210B752500752400752300802EB42A04EC
:20012B00D2018005B43224C2010525E525B40106A20192008015C394075009A201E5243340
:20014B00F5248007A201E52333F523D083D082D0D0D0E032010002000300040005000600C2
:20016B000700080009000A000B000C000D000E000F00100011001200130014001415001678
:20018B0000171A181A191A001B001C001D1F1E1F001F002000212322232B242B2500262859
:1A01AB00272800280029002A2322232C002D302E302F300031003200222B12
:00000001FF
